:020000040000FA
:020000000628D0
:02000800E82AE4
:04000C0003139F013A
:1000100083169F0183128B0100008B1700000B17C2
:1000200083160C14831283168113E0308500003090
:100030008600831286018501900100009015000062
:100040009014000010148316811200008111F83002
:100050008105073081048312A301A401A50180302A
:10006000A600FF30A800A901AA01AB01AC01AD01B7
:10007000AD0AA1013F213C211230A3000530A400AC
:100080000730A5004F280130392208303922C52217
:1000900003303922053039220130E0214328A808F5
:1000A000031D5628A1010230E0214F282608A70091
:1000B0000030210203197E2001302102031987201C
:1000C0000230210203198C20033021020319B620CB
:1000D000043021020319DB20053021020319FF201F
:1000E00006302102031988200730210203198A20D3
:1000F000A00101302102031DE7214F287221232195
:1001000005303102031D08000230A10008007C29DF
:1001100093210800A2210800FF30A7000F30A8009B
:100120002C080339013EA2001330A9000630AA00B2
:100130001930AB00A203031908001530A9000930DB
:10014000AA001530AB00A203031908001930A9005A
:100150000A30AA001330AB00A203031908000A30CA
:10016000A9000F30AA000A30AB0008005921350859
:10017000A900AA01AB012C080739FF300319AA0016
:100180000319AB00A01C080000303202031D080058
:10019000043031020319A30A013031020319A30309
:1001A000183023020319A301FF302302031D0800A6
:1001B0001730A30008002408AA00A901AB012C08ED
:1001C0000739FF300319A9000319AB00A01C080070
:1001D00000303202031D0800043031020319A40A62
:1001E000013031020319A403063024020319A401CB
:1001F000FF302402031D08000530A4000800250874
:10020000AB00A901AA012C080739FF300319A90086
:100210000319AA00A01C080000303202031D0800C8
:10022000043031020319A50A013031020319A50374
:100230000A3025020319A501FF302502031D08001D
:100240000930A5000800003031020319080006300B
:10025000310203193029033031020319362908000D
:10026000A60A003026020319A6090800A603FF30DB
:1002700026020319A60908001030B0000800C0309B
:10028000AE000330AF00A50A0A302502031D56292F
:10029000A501A40A06302402031D5629A401A30ABD
:1002A000572118302302031D5629A3010800080016
:1002B0000800A0110C3023020318A0152308A01970
:1002C000F43E03190C3EB400B5000130B3000A300F
:1002D0003402031CB30134083318F63EB400A019ED
:1002E0003516080059213508A9002408AA00250858
:1002F000AB00AC192B1608005921330839223408F9
:100300003922C5222408392225083922DE220A3062
:10031000A01D0B3039220C303922DE22DE22DE22F3
:10032000DE22DE2208002C081F39AB002C0E0E390D
:10033000AA000310AA0C2D18AA1503102D0C1F39A2
:10034000A90008003108AB0032080F39AA00320EAC
:100350000F39A90008000509E0390319DA29B600A8
:100360008030A800B60E0310B60C31083602031D0B
:10037000D529B20AA01402303102031DC929043064
:100380003202031DC929A10A083021020319A10163
:10039000201502303102031DD42910303202031D12
:1003A000D429A101A801201508003608B100B20126
:1003B000A0140800B108031DA014B201B101080087
:1003C000A2002010201CE229A20BE12908003422FF
:1003D0000508F83906388500290813220508F83978
:1003E000053885002A0813220508F83903388500E6
:1003F0002B081322342208002608003CA20000002B
:1004000000000000000000000000000000000000EC
:1004100000000000000000000000000000000000DC
:10042000A20BFF290800B700B801B80A371C1A2A26
:1004300038088604B901B90A27083902031C1B2AA7
:100440003809860500000000B90F222A0310B80DF4
:100450000310B70CB81E162A08000530B9000000BA
:100460000000B90B2F2A080007308504E03086050C
:100470000800BA00DE22BA080319662ABA03031973
:100480006D2ABA030319742ABA0303197B2ABA0323
:100490000319822ABA030319892ABA030319902A75
:1004A000BA030319972ABA0303199E2ABA03031938
:1004B000A52ABA030319AC2ABA030319B32ABA034B
:1004C0000319BA2ABA030319C52A08000E30CC2230
:1004D0001130CC220E30CC2208001230CC221F303A
:1004E000CC221030CC2208001930CC221530CC227E
:1004F0001330CC2208001530CC221530CC220E301F
:10050000CC2208000730CC220430CC221F30CC2271
:1005100008001730CC221530CC220930CC2208003C
:100520001F30CC221530CC221D30CC2208000130E7
:10053000CC220130CC221F30CC2208001F30CC222C
:100540001530CC221F30CC2208001730CC221530B9
:10055000CC221F30CC2208001F30CC220530CC2208
:100560000230CC2208001E30CC220530CC221E30B6
:10057000CC2208001F30CC220230CC220430CC2206
:100580000230CC221F30CC2208000030CC220A30AE
:10059000CC220030CC220800BA00DE220508073841
:1005A000063985003A0886008030BA000000000055
:1005B00000000000BA0BD62A86010800FF30BB00FD
:1005C00000000000000000000000BB0BE02A080053
:1005D00000308E00F8308F002014A808031DA803F7
:1005E000AC0A0319AD0AAE032E09031DFC2AAF03A2
:1005F0002F09031DFC2A3F21B003300903193C21B8
:06060000AB210C10090003
:02400E00103F61
:00000001FF
